:020000040800F2
:10500000A01A0020D5500008A5860008B57D00082C
:105010000000000000000000000000000000000090
:1050200000000000000000000000000045900008A3
:105030000000000000000000998E00084191000867
:10504000E7500008E7500008E7500008E750000864
:10505000E7500008155B0008E7500008E75000081B
:1050600000000000E7500008515A0008E75000080F
:10507000E75000088D82000800000000E75000089B
:1050800000000000E75000080000000000000000E1
:10509000E750000800000000E7500008E750000853
:1050A000E7500008E7500008E7500008299A000878
:1050B000E7500008E7500008000000000000000072
:1050C0000348854600F060FC00480047F9A7000847
:1050D000A01A00200448804704480047FEE7FEE786
:1050E000FEE7FEE7FEE7FEE7DD910008C15000089D
:1050F00030B50B46014600202022012409E00D4670
:10510000D5409D4205D31D469540491B25469540F7
:1051100040191546521E002DF1DC30BDF0B51FB40C
:105120000646002082B005464024019100901BE015
:10513000019922460F46304600F04EFB049A059B2B
:10514000801A994110D310461946224600F034FBCC
:10515000361A8F410197224601200021009F00F05E
:105160002BFB38184D4100902046641E0028DFDCE0
:10517000019B00982946324607B0F0BD03460B4319
:105180009B0703D009E008C9121F08C0042AFAD2FD
:1051900003E00B780370401C491C521EF9D2704783
:1051A000D2B201E00270401C491EFBD270470022BF
:1051B000F6E710B513460A4604461946FFF7F0FF16
:1051C000204610BD30B504460020034600E05B1CBD
:1051D000934203D2E05CCD5C401BF8D030BDF8B503
:1051E00002464A40D40F42004B0052085B089A42E4
:1051F00002D20246084611464A0023D0C30D4A0097
:10520000DDB2120EAD1A202D35DA49020126490A07
:10521000F6058A19002C00D0524220214F1B11465E
:10522000B9402A411018C20D9A4221D0002C17D043
:10523000012D08DCDA05801AD20F8019D207DBB203
:1052400000F0F6FAF8BDDA05801A012340001B06CB
:10525000C01880185A428018CA0F1043490007E04E
:105260004908C2071143DA05801A801940088018DE
:1052700000F0D6FAF8BD61000122511A001BF7E7D1
:105280000122D2075140AAE70122D2075040A6E7E7
:1052900070B502464A40D50F40004A00ED0740086D
:1052A0005208002814D0002A12D0C40DD30D410298
:1052B0000120C0055202490A520AE41A09181218BC
:1052C0007D34914201D3641C00E04900002C01DAD6
:1052D000002070BD0023914201D3891A0343400886
:1052E00049000028F7D100290AD0914202D10121BA
:1052F000C90705E0914201D2012101E00121C94322
:10530000E005C018401900F08BFA70BDF0B50746F3
:105310000846584087B0C00F049048000E46590018
:1053200040084908BC1A884105D2384631461E4615
:1053300017460B4602465800400810434CD0300D2B
:10534000039040055900400D490D0590401A029008
:10535000402872DA18030121000B09050843019067
:1053600004980092002805D00199524200208841FB
:1053700000920190029840210A1A0199009800F0C9
:105380001BFA05460C466B4607CB00F036FAC019EF
:105390007141039A0E0D0023D71756401A467A40E2
:1053A000164344D0049A002A2DD0029A012A039A67
:1053B00015DC1205C01A914101263605001C714109
:1053C000D20F059ED2070093019202962A462346E9
:1053D00000F074FA07B0F0BD38463146FAE716051A
:1053E000224A0F46B218C01AB74101210905001C14
:1053F0004F4100187F41114618187941E20F1043C0
:105400006D19644113E0E2076D0815436408C20793
:105410001443039A01261205C01A91413605001C57
:105420007141CE07400830434908C01851412A460F
:10543000234600F036FACDE7FFE70498012240004A
:10544000C117121A00238B4104983146C417381A29
:10545000A141EEE730B40124E407634030BC55E7D6
:1054600030B40124E407614030BC4FE70000E0FFA6
:10547000F0B51FB488B00B990998002448400999E9
:10548000C00F490049080991C0070B9900904900D5
:1054900049080B9109990898A64608431CD00B9916
:1054A0000A98084318D0099801244000420D48008A
:1054B000410D099824050003000B204309900B9827
:1054C0000003000B20430B9050181C494018002289
:1054D00001901446104605E0002001460DB0F0BDD5
:1054E000032801DA034600E003239C46C11A0AAEF2
:1054F0000AE05F0008ADED5B4F00F75B7D430027DE
:10550000AA187C41491C5B1E6145F2DD410004ABD9
:105510005A522104120C0A43240C401C0828DFDBD9
:10552000019802900099704601910090059B049AA1
:105530000799069800F0C2F9D0E700000DFCFFFFC4
:10554000F0B50C465C4085B0E40FE40703944C00D2
:1055500000266408590094464908024602962243F0
:1055600021D062460A431ED06200570D4A000E0346
:105570002303550D012402462C492405781B1B0BDF
:10558000360B401823432643614600901C46501AB0
:10559000B44103D30098401C009002E09218009898
:1055A0005B41002803DA0020014605B0F0BD002071
:1055B000012109050746864611E064461D46141B75
:1055C000B54106D36546521BB341744607430C43AD
:1055D000A646CD0740084908284392185B41054676
:1055E0000D43EAD11046184313D060461946504087
:1055F0007140084306D06046101AB34106D201221A
:10560000002306E000220123DB0702E00122D2434F
:105610005310009874460105381C6141029C039D9B
:105620000019694100F03DF9BFE70000FD030000EB
:10563000C217C10F504010B54018CA079623002169
:1056400000F0F6F810BD10B500229623114600F0C8
:10565000EFF810BD0EB5C217C10F5040CA07401871
:105660000021054B0293019200910A460B4600F07F
:1056700025F903B000BD0000330400000EB5054954
:105680000291002100910A460B46019100F016F9A3
:1056900003B000BD33040000410040020122400A73
:1056A000D205090E80187F2901DA0020704796295B
:1056B00003DC9622511AC8407047963988407047DB
:1056C00070B5CD0F4A0009030123090B1B051943CF
:1056D0000B4BED070024520D9A4201DA002070BDF9
:1056E000074B34339A4203DC9A1A00F075F802E053
:1056F0000449511888402C43F1D0404270BD00004D
:10570000FF030000CDFBFFFF4A0009030123090B43
:105710001B051943094B10B5520D9A4201DA0020BE
:1057200010BD064B34339A4203DC9A1A00F054F849
:1057300010BD03495118884010BD0000FF03000050
:10574000CDFBFFFFC20FD207400040080BD0C10DB8
:105750000723DB01C91840020905400A1143C208AA
:10576000400711437047002001467047CB0FDB070D
:10577000490010B5490802460A4307D00A0D07241C
:105780000903E401090B121B002A01DC002010BDF3
:10579000C900440F0C43C100E018D205801800F086
:1057A0003FF810BD0122D207002800DB101A0029A3
:1057B00000DB511A8142704710B5202A04DB0146F4
:1057C000203A9140002010BD914020239C1A0346AE
:1057D000E3401943904010BD10B5202A04DB084671
:1057E000203AD040002110BD0B46D340D0402024A9
:1057F000A21A91400843194610BD10B5202A06DBB5
:10580000CB170846203A1041C1170B4306E00B4660
:105810001341D0402024A21A91400843194610BDDC
:10582000002904DA401C490001D1400840007047BB
:1058300070B40024050C05D11024000402D1002905
:1058400021D01124050E01D100020834050F01D129
:105850000001241D850F01D18000A41C002801DB5C
:105860004000641C002908D020252E1B0D46F54061
:10587000A14000D001212943084301061B1B000A57
:10588000DB1D02D5002070BC7047DB05181880189E
:105890000029F8DA401C4900F5D170BC40084000EE
:1058A000704710B5002B08DA0024401C61419218A3
:1058B0005B411A4301D14008400010BDF0B51FB450
:1058C00082B005460C0003D0084604F06BF902E0F4
:1058D00004F068F920300246009021462846FFF780
:1058E0006BFF049B059A04460F4618431143084377
:1058F00014D0184610431BD0009840210A1A1846AD
:105900000599FFF769FF05460E46009A0599049828
:10591000FFF752FF084305D0012004E02046394636
:1059200007B0F0BD0020C11705430E432C43374399
:1059300000990E986305401A7905E40A00220C4389
:10594000FD0A0A3002D500200146E9E701051019D9
:1059500069410C9C0D9D00196941FFF7A2FFDFE72B
:1059600010B5002904DB0124E40740428C412146A4
:10597000002B04DB1C460123DB075242A341994262
:1059800000D1904210BD0000064C0125064E05E0F6
:10599000E36807CC2B430C3C98471034B442F7D350
:1059A000FFF792FB84AB0008A4AB000838B50446AF
:1059B000064805490068FFF79BFB604300E0401E76
:1059C00000900028FBD138BD40420F00F8000020B5
:1059D000F8B50446006881688907890F012902D15A
:1059E0000168C90722D18168114A1026114001259A
:1059F00000290ED18168294381600120FFF7D6FF7D
:105A000000F0AAFF07460CE000F0A6FFC01B0A2822
:105A100007D9606D30436065A06D2843A065012003
:105A2000F8BD20680068C043C007EDD10020F8BD74
:105A30001700008010B500231A4603E0845CE318C9
:105A40009BB2521C8A42F9D3D84380B210BD0000E9
:105A500010B5034800F036FD024800F033FD10BDDC
:105A60003C160020F415002030B5446C1C252C4059
:105A70000125A540046C6560046863608368102B91
:105A8000036803D099600068C26030BD9A60006806
:105A9000C16030BD10490120487202205E31487259
:105AA00003203C39487204200E3948720A4B0B49D6
:105AB0005A1C0878587149789971233318715971B3
:105AC000203318775977107551751A461E321075A4
:105AD00051751076517670472C110020E00000209F
:105AE00010B503F085FA202003F020FB012004F01C
:105AF00009FC002003F01AFB044804F0A7FA04484C
:105B000004F050FD002004F085FD10BDA800002029
:105B10008380000070B505200121000700F010FF10
:105B200000240D4D002800D02C6002210B4800F00D
:105B300007FF002808D10A482C6000880A21484342
:105B40000849088003F082FF012000F031FE0220A6
:105B500000F02EFE70BD0000F00000200004005098
:105B6000CE000020DE0000207047000010B508497C
:105B700000224A6107494B684C1523434B604B6830
:105B8000082423434B60C009C001026010BD00001F
:105B900084160020002002407FB500250C460646F2
:105BA000039500F0D5FDE009029003A90196009548
:105BB000684600F065FD002804D000F09DFD00203F
:105BC00004B070BD00F098FD0120F9E710B5002386
:105BD00002E0C45CCC545B1C9342FAD310BD0000BD
:105BE00010B5214A00219069C305204804D54169B8
:105BF000022319434161911593699B0505D54369BA
:105C00000124234343616302194393695B0505D56E
:105C10004369082423434361E301194393691B0546
:105C200005D54369042423434361630219439369FF
:105C30009B0405D543691024234343616302194340
:105C400093699B0304D5446920231C434461194391
:105C50009369DB0305D54369402423434361A002D4
:105C60000143916110BD0000002002408416002015
:105C700070B5054600F070FE0646184C0AE0681C38
:105C800008D0002D04D000F067FE801BA84201D987
:105C9000032070BDA069C007F1D1A069800701D5BC
:105CA0000220A061A069C00511D4A06980050ED4AE
:105CB000A06940050BD4A069000508D4A069800440
:105CC00005D4A069800302D4A069C00303D5FFF7FF
:105CD00087FF012070BD002070BD00000020024041
:105CE000F8B51746002605460C4600F031FD09E0E0
:105CF00029460220226800F00DFD002804D1241D51
:105D00002D1D361DBE42F3D300F0F6FCBE4201D27B
:105D10000020F8BD0120F8BD10B50849024600205A
:105D2000054B497905E044001C5B944203D0401CBC
:105D3000C0B28842F7D310BD6E1200204800002088
:105D400010B5094800F0C6FF80B2FFF797FC074A7C
:105D5000074BFFF78DFB0022064BFFF7F1FBFFF728
:105D6000D3FC80B210BD0000B0140020F853E3A5AE
:105D70009B843E4000408F40F8B5414CE0790028BC
:105D800001D0002000E00120E0713D493D48CA7982
:105D90000275097A41753C490A780276497841765C
:105DA0003A48017837481330017005214172962036
:105DB00004F0E8FB4B20C00004F0FEFB3149002258
:105DC00013310C2004F0C8FC00210C2004F0D6FC98
:105DD000022004F027FC2E4D00210F2004F04CFB84
:105DE0002842E062F8D0E06A411C3BD0294E2A4F9D
:105DF000400439D58122D20100210F2004F081FC1A
:105E00000021102004F038FB41061E48490E0022F4
:105E1000633004F067FB1B4D6335687A052820D199
:105E200002221949681DFFF7CDF9002819D1A87A77
:105E3000607113480422691C4030FFF79FF9206C01
:105E400000F02EF860836079294642000B31084645
:105E50007330FFF793F9608B318848433880022014
:105E60002070F8BD02F042FC0C480188608B0546AA
:105E7000FFF73EF93088414339806D1E6583F8BDD8
:105E8000480000208D110020E0000020BE0000200E
:105E900000D02724C8000020C6000020CA0000202F
:105EA00010B504460E4800F015FF0E49C006C00E9E
:105EB000098805E02246C240D2070FD0401CC0B27C
:105EC0008842F7D3012005E02246C240D20705D020
:105ED000401CC0B28842F7D3491EC8B210BD0000B2
:105EE000B0140020CA00002010B5084800F096FA4F
:105EF0000A21064800F032FA044800F01DF9800536
:105F000003D5024800F01AF980B210BD54140020E5
:105F1000F8B52F4D00220121284600F016FDFFF7AD
:105F2000E3FFFFF790FB2B4E3146FFF7B1F92A4C08
:105F30000122A0601146284600F007FD2749A0680D
:105F4000002588423EDB2078254F002815D025709B
:105F5000FFF7CAFFFFF777FB3146FFF799F9A0601B
:105F6000FFF7F0FB00223B46FFF774FA00221D4BBF
:105F7000FFF77EFAFFF7FAFB6060A068FFF7E2FB2D
:105F800000223B46FFF766FA174A184BFFF770FAF4
:105F900006460F466068FFF7D5FB134A144B524282
:105FA000FFF766FA32463B46FFF7B0F9FFF7DEFB34
:105FB00010496060884201DD616004E0FF21C9058D
:105FC000C84200D365606068FFF766FBC0B2F8BDE9
:105FD0000004005000401B442400002000006040EA
:105FE00000000C4000E064403333333333B33040BF
:105FF000CCCCEC3F0000C842F8B50546044640351D
:10600000287C0026012808D0012028742068816897
:106010008907890F01290ED101E00220F8BD01682E
:10602000C90708D0606D2021084360650126002063
:1060300028743046F8BD616DFF220132914302227F
:1060400011436165C1688907890F0091C16889089A
:106050008900C1602068816892071143816000F067
:106060007BFC07460EE000F077FCC01B0A2809D92C
:10607000606D022188431021084360650020287468
:106080000120F8BD206880680028ECDB2068C1682A
:10609000009A1143C160606D80088000401C6065FB
:1060A000C5E70000F8B506460D464036317C0129AB
:1060B0000DD00121317401688A68520709D5416DFC
:1060C000202211434165002030740120F8BD0220D8
:1060D000F8BD174B6A68D80547109A42154C8A6A72
:1060E0002B6812D05B035B0B1A438A622968490351
:1060F00005D5A1680143A1600A20FFF757FC286875
:10610000800312D5A06838430EE05B035B0B9A4313
:106110008A622968490302D5A1688143A160286881
:10612000800302D5A068B843A06000203074F8BD99
:106130000110000000270140406D70470068006CAE
:106140007047000070B5040006D0606D264600253B
:106150004036002802D006E0012070BDA5653574E8
:10616000204600F0D3F8606DC00603D4216888682B
:10617000400705D5606D1021084360653574EBE775
:10618000606DFF22013290430222104360658868EF
:106190008207920F5B48012A02D10A68D2072BD1ED
:1061A000032362689B079A4205D05B429A4202D061
:1061B0005B009A4209D10A69920092080A6121683B
:1061C0000A6963681A430A610CE00A69920092083E
:1061D0000A6181680F22920491438160816862683C
:1061E000114381602168CA6818239A43CA602168F4
:1061F000CA68A3681A43CA608168012252069143A3
:1062000081608168A28E5206114381602068816896
:10621000C90004D4816801221207114381602068FB
:10622000C168394A1140C1602069E168022825D05F
:1062300000200143204620300278037B52035B009C
:106240001A431143226B1143A26992031143E2697D
:10625000D20311432268D3681943D160616A0A46A8
:10626000FF3AC23A05D0A26A11432268D3681943A3
:10627000D16042780121012A02D00BE00420D8E746
:106280000078002823D0606D202210436065A06D47
:106290000843A065E06B012820681FD00169C90789
:1062A00003D0016949084900016120684169C908B2
:1062B000C900416120684169A26B11434161A56534
:1062C000606D80088000401C6065002070BD206803
:1062D000C26801231B041A43C260DBE70269FF2383
:1062E0009B009A43026120680269236CA66C1A43E2
:1062F000636C33431A430261206802690A430261F6
:10630000D3E70000002701401902FEFF10B586B058
:10631000044614216846FEF74AFF0E492068884269
:1063200016D10D48416B421511434163C16A0122E8
:106330001143C162C06A6946104005900220009076
:1063400003200190002002900520000700F03CFA95
:1063500006B010BD0024014000100240F8B504460C
:106360004069254640350E4608280BD02068C06895
:10637000C00709D0606D20210843606500202874A3
:106380000120F8BD082700E00C2700F0E5FA009096
:1063900011E0701C0FD0002E05D000F0DDFA00993E
:1063A000401AB04207D9606D04210843606500209F
:1063B00028740320F8BD206800683842E9D0606D79
:1063C00001214902084360652068C16809058A0FF8
:1063D0000C21002A1BD12022125D002A17D102684D
:1063E000120714D5826853070122002B08DB43688B
:1063F0008B434360606D130298431043606506E071
:10640000606D202318436065A06D1043A065A069EE
:10641000002801D1206801600020F8BD70B5044655
:10642000216800208968490721D425464035297C08
:1064300001291CD001212974E169012904D02046D9
:10644000FFF7C6FA002811D1616D0A4A1140FF22F8
:106450000132114361650021A165297422681C2164
:10646000116021688A6804231A438A6070BD022083
:1064700070BD0000FEF1FFFF70B500240146203121
:106480004A79022A03D00421C163012418E002687A
:1064900013680E25AB431360026813685B085B004A
:1064A0001360436C1C221340012215469D40036C6F
:1064B0005D604A7100220A71816B002900D0884713
:1064C000204670BDF0B4016C0D6801680C68466C24
:1064D0001C2304221E401746B7402F420ED06707E8
:1064E0000CD50C68A40602D40C6894430C60416C73
:1064F00019408A40016C4A60016B1AE00227B740DC
:1065000002462F402032002F17D0A70715D50C6860
:10651000A40605D40C680A25AC430C600121517116
:10652000446C02211C40036CA14059600021117190
:10653000C16A002918D0F0BC08470827B7402F428D
:1065400012D0240710D50C680E25AC430C60446CA7
:1065500001211C400B46A340046C6360C163517170
:1065600000211171416BE4E7F0BC704770B5040085
:106570003CD01F48256814212818FEF7B9FD80007B
:1065800060641C482064022120462030024641718C
:1065900029681948E3680140A068666918432369BF
:1065A00033431843A3691843E3691843236A184324
:1065B000084328600121A0688903884210D00D4853
:1065C0008030836A656C1C210D400F26AE40B343BA
:1065D0008362656C63680D40816AAB400B438362E4
:1065E0000020E06301215171107170BD012070BD68
:1065F000F8FFFDBF000002400F80FFFFF8B5044622
:106600008C46203001790025012909D00126067128
:1066100041790027012905D0077102252846F8BDD8
:106620000220F8BD02214171E76320680168490832
:106630004900016061462046FFF716FA206B0028EA
:106640002068016801D00E2205E004229143016018
:10665000206801680A221143016020680168314303
:106660000160DBE770B5044600F076F90546601C72
:1066700000D0641C00F070F9401BA042FAD370BD3A
:10668000F8B51A4E0546307C0F46012807D0012088
:1066900030741748FFF7ECFA010002D021E0022025
:1066A000F8BD0020C04338606C6814E02046FFF756
:1066B0005DFA0F48FFF7DCFA01460E4842680823EE
:1066C0009A434260426843159A434260002901D0D0
:1066D0003C6006E08034A8686A68C0018018A04267
:1066E000E4D8002030740846F8BD0000841600206D
:1066F00050C30000002002400548416802221143B7
:106700004160416801221143416000207047000050
:1067100000200240F8B50C4C1646207C0F4601289C
:1067200008D0012020740948FFF7A2FA00250028AC
:1067300002D006E00220F8BD65613E600348FFF725
:1067400097FA2574F8BD00008416002050C300009D
:1067500011484168C9070BD0EFF3108172B60F4A98
:10676000C2600F4AC26081F310884168C9070ED128
:10677000416889070DD5EFF3108172B6094A0261AD
:10678000094A026181F310884068800701D5012021
:10679000704700207047000000200240EFCDAB8919
:1067A00005040302BFAE9D8C16151413704700003C
:1067B00010B504494A69024202D04861FFF7F6FF6A
:1067C00010BD000000040140F8B500230124A2E040
:1067D00027469F403A4070D04D68022D01D0122DBF
:1067E00014D1DD08AD002D1800952D6A5E07AC466A
:1067F000F50E0F26AE46AE406546B543AC460E6973
:106800007546AE4065462E43009D2E624D68012DB3
:1068100005D0022D03D0112D01D0122D16D185687F
:106820000326AC465D00AE46AE406546B543AC4679
:10683000CE687546AE4065462E43866046680D7943
:10684000BE43ED06ED0F9D403543456006685F0091
:106850000325BD40AE46AE430D79B446AE07B60F34
:10686000BE4065462E430660C6687546AE438D68D9
:10687000BD403543C5604D68ED004BD5294D6E6B6D
:1068800026436E639E08284DB6007519AC46AD6868
:106890009E07360F0F27B740BD4305273F07B84275
:1068A00001D1002715E0214FB84201D1012710E0A6
:1068B0001F4FB84202D102270BE02BE01D4FB84218
:1068C00001D1032705E01C4FB84201D1052700E0A4
:1068D0000627B7402F436546AF60184D2E684F68B6
:1068E0009643FF0300D516432E606E684F689643AB
:1068F000BF0300D516436E60AE684F689643FF0233
:1069000000D51643AE60EE684F689643BF0200D5CF
:106910001643EE605B1C0A681546DD4000D057E761
:10692000F8BD0000001002400000014000040050CB
:1069300000080050000C0050001C005000040140F2
:106940000069084000D001207047002A01D0816111
:10695000704781627047000001480068704700007E
:10696000F400002002480168491C016070470000E3
:10697000F400002010B508480024016840221143AB
:106980000160204600F00AF8002801D0012401E04F
:1069900000F0CCF9204610BD0020024070B505463D
:1069A00009487D210024C9000068FEF7A1FB00F022
:1069B00061FE002801D0012404E000222946501E77
:1069C00000F0D4F9204670BDF800002070477047F1
:1069D000F8B53A4C01266078401C6070E670208C57
:1069E000401C2084608902F06BFB354FF888FEF76D
:1069F0002AFE3449FEF74CFC334D00902968FEF71F
:106A0000EEFB2860A16AF005814203DB0098FEF7E7
:106A10003BFCA06202212D48FFF792FF002808D01E
:106A20000020E0622A492F682A488F4227DD06703D
:106A300027E0F888FEF707FE2249FEF729FCE16A05
:106A4000FEF7CDFB2449E0628842EBDBE0790028C9
:106A500013D000211A484030818004F003F801214E
:106A6000002289021948FFF770FF7D200001FFF71F
:106A7000F9FD1B491948C860D4E70121EAE7002164
:106A80000170207A401EFEF7D3FD3946FEF78AFEDC
:106A900006D82079002803D01248C1793143C1714A
:106AA000207AFEF7D0FD2968FEF77CFE04D220791B
:106AB000002801D003F03AFFF8BD0000BC00002020
:106AC0002C0D002000007A44F0000020000400504B
:106AD000000040404E0000200000A0400400FA05E5
:106AE00000ED00E0A0110020704770B505000DD04A
:106AF00002202C462034A073284601F0CFFB284604
:106B000000F0BEF80020A073607370BD012070BD5E
:106B10007047704710B5044600680168C943C9074B
:106B200008D18168C943C90704D1012141602046C9
:106B3000FFF74EFF20680168C943890708D48168C0
:106B4000C943890704D4022141602046FFF73EFF74
:106B500020680168C943490708D48168C9434907C7
:106B600004D404214160204600F0DEF8206801686A
:106B7000C943090708D48168C943090704D4082117
:106B800041602046FFF7B0FF20680168C943C9068D
:106B900008D48168C943C90604D410214160204645
:106BA000FFF715FF20680168C943890608D481688A
:106BB000C943890604D4202141602046FFF7A9FF7C
:106BC00020680168C943490608D48168C943490659
:106BD00004D4402141602046FFF79AFF10BD000019
:106BE000F8B5040005D025462035A87B002802D042
:106BF00006E00120F8BD00206873204600F052F83E
:106C00000220A8732068C26884466368012B04D000
:106C10000120A16AC005814201D11E20824315488E
:106C20006169814201D0144802401448A6680240BC
:106C300018463043676A266A3E433043A66A3043AB
:106C40001043012B03D00122D205964203D12369C0
:106C5000E2681A431043074A914205D0A2691143E2
:106C6000E2690243084610436146C8600120A873E8
:106C70000020F8BDFFFF00003F1FFFFFF8F119FFE4
:106C800010B500680549884207D10548816B490065
:106C9000490881630D2000F055F810BD007C0040CC
:106CA0000010024010B50068084988420CD108481D
:106CB000816BC20411438163002201210D2000F089
:106CC00055F80D2000F048F810BD0000007C004091
:106CD000001002400068C0697047000070B50224CF
:106CE000034620339C730F4C2568E604354325602A
:106CF0000468E568B6123543E5600568AE680124AE
:106D00002643AE6005682E6926432E610568A96199
:106D100001684A61006801690422114301619C73A2
:106D2000002070BD00040140704700000448416B22
:106D3000012211434163816B020411438163704757
:106D400000100240C106C90E0120884001490860B8
:106D50007047000080E100E0C106C90E01208840B4
:106D6000014908607047000000E100E010B501F043
:106D70009BFC10BD02494A6882434A60704700008C
:106D8000007000400248016882151143016070479D
:106D90000070004002494A6802434A6070470000A0
:106DA0000070004005480168022211430160044858
:106DB000016904221143016130BF70470070004037
:106DC00000ED00E00A4B1A689208920002431A6034
:106DD00008480369042213430361012906D040BF18
:106DE00020BF20BF016991430161704730BFF9E7BF
:106DF0000070004000ED00E0F8B504460078544D06
:106E0000800672D5524E0027403EB06BC00004D4BD
:106E1000B06BA9050843B06301274E480168C90556
:106E200011D40168821511430160FFF795FD0090B0
:106E300005E0FFF791FD0099401A642837D84548CE
:106E40000068C005F5D532680321090560680A406D
:106E50000140914208D08103890F032904D1316890
:106E6000890301D50120F8BD2A69032109040A40DC
:106E700022D0084090421FD0207880061CD5286977
:106E80002A6988430121C9040A432A612A698A437D
:106E90002A612861C0050FD5FFF75EFD009008E06C
:106EA000FFF75AFD0099411A2B48814201D903206E
:106EB000F8BD28698005F3D561688803800F032831
:106EC00005D132680005824301400A4332602869D7
:106ED000032261681204114008432861002F04D086
:106EE000B16B012000078143B1632078C00705D052
:106EF000E868A168800880000843E860207880077F
:106F000005D5E8680C218843E1680843E8602078EB
:106F1000400706D5E86803218902884321690843B0
:106F2000E8602078000706D5E86803210903884354
:106F300061690843E8602078000606D5E868032107
:106F400089048843A1690843E8600020F8BD000077
:106F5000401002400070004088130000F8B50E4653
:106F600005007DD053480068C007C00FB0420AD268
:106F70005048016849084900314301600068C00772
:106F8000C00FB04271D128784B4C800705D5E0681E
:106F9000F0218843A9680843E0602878C00752D0F0
:106FA0006868022817D0032818D02168012818D053
:106FB0008905002959DAE168890889000143E160FF
:106FC000FFF7CAFC69680746022912D003291CD0C2
:106FD000012926D033E021688903EAE72168890185
:106FE000E7E74907E5E7FFF7B7FCC11B33488142F4
:106FF00023D8E0680007800F0228F4D123E0FFF7D0
:10700000ABFCC11B2D48814217D8E0680007800FF8
:107010000328F4D117E0FFF79FFCC11B27488142EA
:107020000BD8E0680007800F0128F4D10BE0FFF7D0
:1070300093FCC11B2148814201D90320F8BDE068BF
:107040000007800FF3D11B480168C907C90FB1427F
:107050000DD901684908490031430160006800E02A
:1070600003E0C007C00FB04201D00120F8BD28786E
:10707000400706D5E068072109028843E96808430C
:10708000E0602878000707D5E0680721C902884337
:107090002969C9000843E06000F036F8E168084A51
:1070A0000906090F515CC840064908600020FFF737
:1070B00075FCF8BD0020024000100240881300005B
:1070C00062AB0008F8000020044805490068C96860
:1070D000044A4905490F515CC8407047F800002038
:1070E000001002407BAB0008044805490068C968ED
:1070F000044A8904490F515CC8407047F8000020D9
:10710000001002407BAB000810B5184AD1680C2073
:10711000084004280BD0082810D00C2810D0506844
:107120000004410F0120C003491C884010BD1068B5
:10713000C00601D50E4810BD0E4810BD0E4810BD4A
:1071400088020E4B000F185C0902D368890F491C96
:10715000DB0301D5084A05E01268D20601D5044ACE
:1071600000E0044A5043FDF7C3FF10BD0010024089
:1071700000093D000024F40000127A0072AB000800
:10718000FEB505007ED0FE4CE7680C20E66807409F
:107190000120000406402878C00747D0082F05D0FA
:1071A0000C2F0AD101200004864206D120688003FA
:1071B0003CD568680028E5D038E001206968000403
:1071C000814203D121680143216011E0052301229E
:1071D0001B0492049942216802D111432160F1E716
:1071E0008143216021680140009120689043206024
:1071F000686800280DD0FFF7AFFB009005E0FFF7AF
:10720000ABFB0099401A64287AD820688003F6D531
:107210000CE0FFF7A1FB009005E0FFF79DFB009954
:10722000401A6428F0D820688003F6D428788007B4
:1072300055D50923E868042F0DD00C2F01D1002E5D
:1072400009D000283BD02168994301432160FFF712
:1072500083FB064627E02168490701D5002891D025
:1072600061681F22120291432A6912021143616070
:107270002168994301432160FFF746FFE168090651
:107280000A0F00E079E1BF49895CC840BE49086047
:107290000020FFF783FB002872D120E0FFF75CFBA2
:1072A000801B0228B0D820684007F7D560681F21EE
:1072B0000902884329690902084360600FE02068D9
:1072C000400840002060FFF747FB064604E0FFF758
:1072D00043FB801B022897D820684007F7D4287802
:1072E000C0065FD5002F0CD0A869002849D02068BF
:1072F000FF21013108432060FFF72EFB06462DE0F9
:10730000C0E02068800502D5A8690028A7D0606881
:10731000072149038843296A084360606068297F20
:107320000002000A090608436060286A410B012038
:10733000C003491C8840E16809060A0F9149895C2D
:10734000C840914908600020FFF728FB002817D1AA
:1073500028E0FFF701FB801B0228A3D820688005E6
:10736000F7D56068072149038843296A08436060AC
:107370006068297F0002000A09060843606011E086
:10738000E1E02168FF20013081432160FFF7E4FA4A
:10739000064604E0FFF7E0FA801B022872D8206856
:1073A0008005F7D42878794E000724D5686900282D
:1073B000306910D0012108433061FFF7CDFA009009
:1073C00005E0FFF7C9FA0099401A02285AD8306937
:1073D0008007F6D50FE0400840003061FFF7BCFAA7
:1073E000009005E0FFF7B8FA0099401A022849D842
:1073F00030698007F6D42878400765D500200290D0
:10740000A06BC00006D4A06B012109070843A0634C
:10741000012002905E480168C90511D401688215F7
:1074200011430160FFF798FA009005E0FFF794FA26
:107430000099401A642825D855480068C005F5D53C
:10744000FF20AA680130824203D1316901433161D2
:1074500011E001218902002A07D005231B029A426C
:1074600003D132690A433261EFE732698243326104
:10747000306988433061A86800280FD0FFF76CFAA4
:10748000009007E05EE0FFF767FA0099411A414873
:10749000814257D830698005F5D50DE0FFF75CFAD9
:1074A000009006E0FFF758FA0099411A39488142E6
:1074B00048D830698005F5D40298002804D0A06B24
:1074C000012109078843A063686A002864D00C2F53
:1074D0003ED0012636060228206805D0B043206041
:1074E000FFF73AFA05462FE0B0432060FFF734FA81
:1074F000074604E0FFF730FAC01B022822D82068B4
:107500008001F7D4E96AA86AE2680843296BFD2381
:107510001B049A4311430843E06020683043206015
:10752000FFF71AFA054604E0FFF716FA401B022897
:1075300008D820688001F7D52EE0FFF70DFA401B30
:10754000022801D90320FEBD20688001F5D423E084
:107550000128F8D0E06801210904AA6A014091429B
:107560000BD10F218904EA6A0140914205D1032120
:1075700089050840296B88420ED00120FEBD00001D
:107580000010024062AB0008F800002040100240EA
:1075900000700040881300000020EFE770B5040081
:1075A00007D0002625464035A662687C002802D018
:1075B00005E0012070BD2E74204600F02FF8022057
:1075C000687420680168402291430160A168606886
:1075D00022690843E16811430843616901220843B5
:1075E000A169520211400843E1690843216A084336
:1075F000A16A084321680860A0690421000C0840C2
:10760000616A0843216848602068C169920091431B
:10761000C161666501206874002070BD10B586B038
:10762000044614216846FDF7C2FD104920688842CF
:1076300019D10F48416B821411434163C16A012281
:107640001143C162C06A002110400590E020009003
:1076500002200190032003900291049105206946C5
:107660000007FFF7B1F806B010BD00000030014080
:1076700000100240094910B5401E884201D901207E
:1076800010BD074C60610321081F01F00DF80020B8
:10769000A06107202061002010BD0000FFFFFF0057
:1076A00000E000E0F0B502462032137E012B15D039
:1076B000012717760223537605686C68AB6870263D
:1076C000B4430E68496826438024A34319436E607F
:1076D00000688160577600201076F0BD0220F0BD72
:1076E00070B5040005D025462035687E002802D0FC
:1076F00006E0012070BD00202876204600F00AF840
:1077000002206876211D206801F094FD0120687632
:10771000002070BD00680449884204D10348416BD1
:1077200004221143416370470008014000100240E9
:10773000F8B5054604462035287E012817D00126D5
:107740002E7602206876226890687727FF23B84358
:107750001B02984390600A68502A31D00EDC202A20
:107760004BD006DC002A48D0102A3AD145E002204E
:10777000F8BD302A41D0402A33D136E0602A27D0E4
:10778000702A12D001200003121A2AD0824228D176
:10779000CB684A688968206801F085FD20688168A7
:1077A00001229203114381601BE0CB684A6889681B
:1077B000206801F078FD216888683843886010E00F
:1077C000CA684968206801F0E8FD5021206806E099
:1077D000CA684968206801F0F1FD6021206801F065
:1077E0006DFD6E7600202876F8BDCA68496820686D
:1077F00001F0D3FD40212068F1E711462068EEE753
:1078000010B586B0044614216846FDF7D0FC0D493A
:107810002068884213D10C48C26A02210A43C2621E
:10782000C06A019108400590480300900020029032
:1078300003900620049069460448FEF7C5FF06B091
:1078400010BD00000008014000100240000400507C
:10785000F8B5064604462036307E0D4601280DD088
:1078600001203076022070760427002A08D0042AEE
:1078700016D0082A2AD00C2A4DD137E00220F8BDB4
:10788000206801F023FD206881690822114381618D
:1078900020688169B943816120688169EA6812E0E2
:1078A000206801F02BFD206882690121C9020A438A
:1078B000826120688169012292029143816120687E
:1078C0008169EA6812021143816124E0206801F0B5
:1078D0002EFD2068C26908210A43C2612068C1697F
:1078E000B943C1612068C169EA6812E0206801F00B
:1078F00039FD2068C1690122D2021143C1612068AB
:10790000C269012189028A43C2612068C169EA68AB
:1079100012021143C1610120707600203076F8BD5B
:1079200070B5040005D025462035687E002802D0B9
:1079300006E0012070BD00202876204600F00AF8FD
:1079400002206876211D206801F074FC0120687611
:10795000002070BD704710B504460068012201F098
:1079600095FC206881684907490F062903D0016802
:10797000012211430160002010BD000010B5044633
:107980000068002201F082FC2068016A054A114269
:1079900003D1016849084900016001202034607664
:1079A000002010BD1111000070477047F8B5026843
:1079B0000446D0691168936805072D0F5BD0DD0779
:1079C000ED0FFF2621360E402E4367D0C60706D0A6
:1079D000CE0504D501261662E26F3243E2678707BF
:1079E00002220426002F06DADF0704D027683A6255
:1079F000E76F3743E767470706D5DB0704D02368FF
:107A00001E62E36F1343E367020709D520220A4091
:107A10002A4305D0236808221A62E36F1343E36701
:107A2000E26F002A2FD0800606D5880604D5216E85
:107A3000002901D020468847E06F216889684906FF
:107A400001D4000724D5204601F05EFE206881683D
:107A5000490619D58168402291438160E06E002873
:107A600012D020498163E06EFEF706FD00280AD09F
:107A7000E06E816B06E0850610D58D060ED5216E71
:107A80001CE020468847F8BD2046FFF78EFFF8BD72
:107A90002046FFF78AFF0020E067F8BDC50208D541
:107AA0005B0206D50120000510622046FFF77CFF2F
:107AB000F8BD030605D50B0603D5616E0029E0D19C
:107AC000F8BD4006FCD54806FAD51368204640218B
:107AD0008B431360202161670021616600F069F922
:107AE000F8BD00006596000810B5040003D0606F73
:107AF000002802D007E0012010BD002170200155B0
:107B0000204600F027F824206067206801684908B3
:107B100049000160204601F041FE0128ECD0606A76
:107B2000002802D0204601F07FFC2068416809222D
:107B3000D20291434160206881682A22914381608A
:107B400020680168012211430160204601F0D2FC47
:107B500010BD0000F0B587B0064614216846FDF759
:107B600026FB2C493068884251D12B48416B0122B9
:107B7000920311434163C16A01221143C162C06A89
:107B800000251040059003204002009002200327AA
:107B900001A9A1C104200490052069460007FEF751
:107BA00013FE1F4C1D48A560E56081C48027E56079
:107BB000A7602020256160610002A0611848083C90
:107BC000FEF7D4FC002801D0FDF7CEFFF466A662D4
:107BD000144C1248214614382060032060601020A5
:107BE0000831A1C16561A561E56120462562FEF706
:107BF000BDFC002801D0FDF7B7FFB46600220121CB
:107C00001B20A662FFF7B2F81B20FFF7A5F807B00C
:107C1000F0BD00000038014000100240300002407A
:107C2000F41500203C160020F8B50446806F20288B
:107C30004DD100290BD0002A09D00123A0681B03D5
:107C4000984206D12069002803D1C80701D001203D
:107C5000F8BD25466035287C012838D001202874DD
:107C60005820616502530026E6672220A067E06E77
:107C7000002819D01749C162E16E17480863E16E08
:107C800016484863E06E13468663676D21683A467E
:107C90002431E06EFEF7B2FC002805D01020E0672A
:107CA0002E7420206067D2E72E7420680168FF22BE
:107CB0000132114301602068816801221143816013
:107CC000206881684022114381600020F8BD0220B5
:107CD000F8BD0000C1960008FF96000879960008DC
:107CE00070477047FFB50446406F83B017460D4696
:107CF00020285CD1002D0AD0002F08D0A168C00137
:107D0000814207D12069002804D1E80702D0012070
:107D100007B0F0BD204660300290007C012846D0BC
:107D20000298012101740020E06721206067FEF7BE
:107D300013FE264640360190378277820120A168E3
:107D40000003814202D12069002802D02F4600257D
:107D500011E000270FE000228021204601F032FED2
:107D6000002815D1002F15D02168387888627F1C33
:107D7000708A401E7082708A019B002806980090CD
:107D8000E9D100224021204601F01CFE002808D045
:107D90000320BDE728882168C005C00D8862AD1C9E
:107DA000E6E720206067029900200874B0E702200F
:107DB000AEE7704701490248C160FDE70400FA05DB
:107DC00000ED00E070B501240525E4022D07002236
:107DD00021462846FEF7B9FD002204210948FEF796
:107DE000B4FD0A2002F0EBF8012221462846FEF7F6
:107DF000ACFD0A2002F0E3F8002221462846FEF7F7
:107E0000A4FD70BD0004005070B501240525E402F6
:107E10002D07002221462846FEF797FD0122042166
:107E20000948FEF792FD0A2002F0C9F80122214616
:107E30002846FEF78AFD0A2002F0C1F800222146FA
:107E40002846FEF782FD70BD00040050F1B5002405
:107E50000126F602052725463F070022314638460F
:107E6000FEF773FD0A2002F0AAF8012231463846D7
:107E7000FEF76BFD6006040E04210C48FEF760FD62
:107E8000002801D0641CE4B2052002F098F86D1CB3
:107E9000EDB2082DE1D30098002803D0FFF792FF40
:107EA0002046F8BDFFF7B0FFFAE7000000040050DD
:107EB000F8B5012605270546F6023F0700223146A0
:107EC0003846FEF742FD0024E80901D0012200E017
:107ED000002204210E48FEF738FD6806050E0A2030
:107EE00002F06DF8012231463846FEF72EFD0A20D9
:107EF00002F065F8002231463846FEF726FD0A20DA
:107F000002F05DF8641CE4B2082CDDD3F8BD00007B
:107F10000004005070B50E4C012204212046FEF7EB
:107F200014FD01220526D502360729463046FEF704
:107F30000CFD002204212046FEF707FD0A2002F076
:107F40003EF8002229463046FEF7FFFC70BD0000D7
:107F50000004005070B501240525E4022D0700221D
:107F600021462846FEF7F1FC0B4E00220421304644
:107F7000FEF7EBFC0A2002F022F8012221462846F7
:107F8000FEF7E3FC012204213046FEF7DEFC0A2066
:107F900002F015F870BD000000040050F8B5154D52
:107FA0000024012204212846FEF7CFFC062002F01F
:107FB00006F801220527D6023F0731463846FEF76C
:107FC000C4FC062001F0FBFF07E0641CE4B2FA2CBD
:107FD00003D9FFF7BFFF0120F8BD04212846FEF7B3
:107FE000AFFC0028F1D1002231463846FEF7ADFC47
:107FF0000020F8BD00040050F8B501F0ABFA01F024
:10800000E5FA55480068C069544E554F800700D5C1
:10801000FE60FDF795FE5349534D898F534C00295F
:1080200029D053490A7801218902002A05D0012A62
:108030000ED0022A10D0032A1DD1A08B01282CD0EB
:10804000022818D1444808213C38FFF797FC12E079
:10805000FF22F5329042F0D2A08B01281BD00228DB
:1080600004D008E02846FEF770FC04E03A480821F6
:108070003C38FFF770FC40213B48FEF761FC0025CF
:1080800000282CD03B480560FDF742FF2070A07906
:10809000002804D007E00022E4E70122E2E7012003
:1080A000A07101F0D3FC2078632806D900220821B2
:1080B0002D48FEF74AFC012205E0012208212A484A
:1080C000FEF743FC002201210520C9030007FEF74B
:1080D0003CFC244C4034A08C012803D01CE0A5714A
:1080E0000022EBE724486946088072B680212348C5
:1080F000FDF752FD002804D0022269461F48FDF713
:10810000EFFD62B61EA001F03DFDA58402F0AAFCC1
:10811000642001F04DFFFE60608C012808D11148F9
:108120006584058002F09EFC642001F041FFFE6042
:10813000208C012806D1258402F094FC642001F0F3
:1081400037FFFE600748124A0188914202D1C08879
:10815000002800D1FE60F8BD741500200400FA0567
:1081600000ED00E02C0D002000040050BC000020B9
:108170005A000020F0000020AAAA0000384A000897
:10818000BDF8C8EBC9FDBCB6C4A3CABD0D0A00004A
:10819000AA55000008B53721202000F072F803210D
:1081A000212000F06EF84021222000F06AF808211A
:1081B000232000F066F8AA21302000F062F80C4875
:1081C000018F142901D902210187C9B2322000F0A0
:1081D00058F80121332000F054F85F21202000F0EE
:1081E00050F8684600F006F80A2001F0E8FE08BDE5
:1081F0002C0D002010B501460F2000F021F80028BA
:1082000000D0012010BD10B50446FFF783FE3220D8
:10821000FFF74EFEFFF7C2FEE0B2FFF749FEFFF7A1
:10822000BDFEFFF777FE3320FFF742FEFFF7B6FEF5
:108230000020FFF70BFE0446FFF78CFE204610BD22
:1082400010B50C46FFF7DFFF2070012010BD70B5A0
:108250000D460446FFF75EFE3220FFF729FEFFF7CA
:108260009DFEE0B2FFF724FEFFF798FE2846FFF7D9
:108270001FFEFFF793FEFFF76DFE0A2001F09FFE41
:1082800070BD10B5FFF7E3FF012010BD10B5024827
:10829000FEF740FC10BD0000B0140020FEB50446FF
:1082A000002572B60068394A831804D13849CD6870
:1082B000032189040D4081680191C16800914169E1
:1082C0008669002B08D132484038836AC7043B4393
:1082D0008362836ABB4383620846304348D02B489D
:1082E0002368C34205D12A48C368032292049343FA
:1082F000C360002917D02068026901231A43026174
:1083000020684161FEF728FB0746FEF725FB216840
:10831000C01B0968090703D47D21C9008842F4D92C
:10832000216808204860002E17D0206801690122CA
:108330001143016120688661FEF70EFB7D2706462A
:10834000FF00FEF709FB2168801B0968C90601D4FC
:10835000B842F6D92168102048600C482168C14213
:1083600006D10B48C1680322920491432943C1609E
:108370002068016949084900016121680198886005
:1083800021680098C86062B6FEBD00000084FFBF8F
:10839000401002401CB5002116480091144A01917A
:1083A0000260C1631205426081600722826301227C
:1083B00002610246C16020321170FF235170C23346
:1083C00043628162117301638161042241634261EE
:1083D000C161FDF7B7FE084800908013019069461F
:1083E0000448FDF75FFE00210248FDF705FE1CBDB5
:1083F00000240140541400200200000408B508487D
:10840000016B012211430163006B012110400090B8
:1084100000220A20FEF7AAFC0A20FEF79DFC08BDF8
:1084200000100240F0B587B014216846FCF7BFFE8B
:108430004848C26A04210A43C262C26A0A400592DD
:10844000C16A80273943C162C16A39400591C16A56
:1084500001252943C162C16A29400591C16A0226EA
:108460003143C162C06A2A46304005900520102180
:108470000007FEF76AFA012237493848FEF765FA25
:10848000002237493548FEF760FA9921052000227D
:1084900009020007FEF759FA32480190002405202E
:1084A0006946009502940007FEF78EF910200090AF
:1084B000052069460396019502940007FEF784F9AA
:1084C00005200090112001900294694603942348EE
:1084D000FEF77AF9244801906946009602951F48F4
:1084E000FEF772F9214800900294694601950394C1
:1084F0001A48FEF769F991200002009005200294C5
:108500006946019503940007FEF75EF9E8020090C2
:108510001120019005200294694603940007FEF79C
:1085200053F9402000900194694602940B48FEF7ED
:108530004BF969460948009702950194FEF744F902
:10854000002201210520FEF711FC0520FEF704FCA6
:1085500007B0F0BD0010024001020000000400500E
:108560000C30000000001110000021100832000043
:1085700010B50F4C0D482060FF20053060600020D2
:10858000A060E06020616061E06101212062490239
:108590006062A161A0620720E0622046FEF7FEFF54
:1085A0002068016840221143016010BD0030014085
:1085B000E014002010B58AB00024049405940694B9
:1085C0000794089419480994009401940294164958
:1085D000039401600921846041600461144944618D
:1085E000C160FFF77DF801200003049004A90F4843
:1085F000FFF79EF80D48FFF793F9089408A90B4878
:108600000994FFF74FF8602000900A480190029407
:108610000422694603940548FFF71AF90348FFF757
:10862000EFF80AB010BD0000000801403815002026
:10863000930400004902000000B585B0142168468B
:10864000FCF7B5FD164815490160E121490241607A
:1086500000218160C160016181610C22C1614261C0
:108660000162302141620121090381634900C16334
:10867000FFF73AFA012080020090022001900120C9
:10868000029003200390042004900520694600070F
:10869000FEF79AF801F0D4F905B000BD00380140AA
:1086A00074150020704700008307FF22DB0E9A40FC
:1086B0008907090E994000280BDA0007000F0838D7
:1086C000830808489B001818C36993430B43C36190
:1086D0007047830804489B001B18186890430843A0
:1086E0001860704700ED00E000E400E0BFF34F8F3A
:1086F00004490348C860BFF34F8F00BFFDE7000087
:108700000400FA0500ED00E0F0B58FB0962001F00E
:1087100039FF4B20C00001F04FFFFF4C0025657072
:10872000A07B0C2801D30B20A0730122052051024D
:108730000007FEF70AF9A07B60736071F748A57027
:10874000F74E00783070F748022100783071F64813
:10875000FEF7F6F8002862D00020A179F04E49001B
:108760000843F071A06AF070401CA0626079314645
:10877000B0724200CE310846C338FCF7FFFC062039
:108780007072304613380290217F0175617F417508
:1087900060790022400031460D3001F0DDFF607944
:1087A000002140000D3001F0E9FF022001F03AFF06
:1087B000F5712574A57201202073E572DB48FEF780
:1087C00089FA20840646A5706079FCF757FFD84ADD
:1087D000D84BFCF74DFE01F087FB0022D64BFCF78F
:1087E00095FDFCF791FF0006C10C881980B20121AC
:1087F000C9036084884201D3401A6084CF48606313
:10880000E078401CE070C948FEF764FAE083CC4889
:108810000C90C3484E300B901630019027E2012097
:108820009BE7C248FEF756FAE083C64EC64F21E0EA
:10883000A07A002813D001F066FE039988420ED971
:10884000069988420BD201F035FD2573099801F095
:1088500092FE012001F0E6FE2072A57211E0B348FD
:10886000FEF738FA80B2E083618C884202D3C919DE
:10887000884206D300210F2001F0FEFD3042E06265
:10888000D6D0E06A411C1FD040047DD58122D201A0
:1088900000210F2001F035FF0021102001F0ECFD38
:1088A00041069F48490E002250300A9101F01AFEFD
:1088B000002001F081FE002001F033FE984E50367A
:1088C000707A0728AAD101E0FFF710FF02229F4922
:1088D000701DFCF777FC0028A0D19148503001783A
:1088E0008E480078814299D100273E460DA801F0BC
:1088F00010FE04200DAA390E36020E433902175C11
:108900000F43401EF7D5A764E66400273E46104695
:1089100001F0F1FD04200DA93A0E360216433A0289
:108920000F5C1743401EF7D527656665A1786A4638
:10893000491CA1707A494D310E7916774F796946F5
:108940004F77607B002809D1012275482271898BFD
:10895000CE3001806271029806754775704869468D
:10896000CE300088898B059188427DD10B9878495B
:10897000008A08806A4826464C30808A20836B48EB
:10898000FEF7A8F9F08300E066E1308B7149FF3013
:10899000C33080B2308388420CD9494240186C49B8
:1089A000308308886B4A401C80B20B3208809042AA
:1089B00000D30D806849032008700B98564A8189BE
:1089C0001186C089644B5086903B326B1A601A4600
:1089D000B03AD37C1F073F0F032F00D0B7741A099A
:1089E000F274F57001274C4AB7729186D08670797F
:1089F000FF21913148435749326D593940180104DC
:108A0000C817736D891858410206080A1043534964
:108A1000099040180390192109988902401806907E
:108A20000998B843010E0002F165B0653C48F36C4B
:108A30000A30B26C01F0C8FE3948736D1630326DE1
:108A400001F0C2FE3648F36D1230B26D01F0BCFE8B
:108A50003348082141723149002209780170707948
:108A60002F4980001C3000E09EE001F075FE707917
:108A7000002180001C3001F081FE29492648F77250
:108A8000042251314030FCF779FB3148318B0788A3
:108A90007D20C00078434018B0630D9030480078C6
:108AA000F073009026484038C088FCF7CCFD059054
:108AB0003846FCF7C8FD0599FCF7EAFB7F21C9059C
:108AC000FCF78DFBFCF7E8FD81B22548018000989A
:108AD000401E814201D10120F072B7841420305E23
:108AE000FCF7B8FD07910890F08BFCF7C7FD1D4A15
:108AF0001D4BFCF7BDFC00910A900D98FCF7AAFDF8
:108B0000009B0A9AFCF7A6FC079B089AFCF7FEFB61
:108B1000FCF7D6FDF06329E048000020BE000020ED
:108B2000A0110020BC00002000040050B014002060
:108B3000666666666666E63F00000840A08601003D
:108B40006C0D002000D02724983A0000E00000209F
:108B5000EC000020E70300003013002000AEFCFF13
:108B6000DC000020F853E3A59B843E40BE4800880B
:108B700000F0A6FAF07C002879D00C99098881428F
:108B800075D00C98E17C01801222B8480199FCF75D
:108B9000F5FA0822B549B648FCF7F0FAB349B448EB
:108BA0000A220831303057E10846FDF7B5F8617BFD
:108BB00088420CD30122227162794300521C6271F7
:108BC000AA4A0599CE3AD15202990E754F75A74916
:108BD00003220C390A540B99A64A8B891386870005
:108BE000C989A24851869C38216BC151B038C27CDA
:108BF000A37C1107090F2646994202D9032900D008
:108C0000B274F17C002912D002229B49401DFCF76E
:108C1000D9FA00280BD1012098493074C8710A98FC
:108C20001638C2B2727491480199FCF7A7FA9348BA
:108C3000736D38181630326D01F0C6FD7079002260
:108C400080008E491C3001F087FD70790021800082
:108C50001C3001F093FD0AE0324600210F2001F0A4
:108C600050FD207B002802D0002001F05AFCE18B4F
:108C7000608C814200D2D4E5814A80188142FAD8C2
:108C80008048018888000818E178884200D2A574DD
:108C90007D4A00210F2001F034FDA07860717348F7
:108CA00000260C380078002812D1206CFDF7F8F867
:108CB0000746764801883846FCF71AFA74487F1E42
:108CC0000088414388B268490880678300F0F8F95A
:108CD0000020A073617B22798A1822E0634B0C3B51
:108CE000195C00291BD0A57BB3006D1CA5735F4DDB
:108CF0009C463C3DE9505D4B4500CE3B77005D5BBB
:108D00001833DD5385001A33584F5D5963466C3F65
:108D1000FD50761C3B466033491EF6B21954401C88
:108D2000C0B28242DAD8A078032801D2A07BA07317
:108D300050490022887B48730390401E31E0002197
:108D40002BE04A4C8B006C3CE6581D1906956D686B
:108D5000AE4220DDB646454E4C00B63E365B97002F
:108D6000B446424E3C3EF6590796404E6C3EF55096
:108D700035464A3D67197D884A3E355334467A3434
:108D80001C197A366568F550069B76465E60664625
:108D90007E80079E6660491CC9B28142D1DB521CAD
:108DA000D2B28242CBDB334800214172039C2BE0DC
:108DB0002E4B2E4ACE3B4F00B63AD25BDA531D46BD
:108DC0008A0062351E46AD583236B550314EB54236
:108DD00018D01D469235AD580A2D13D1457A062676
:108DE000AC4675431E461A3EFB18AD191B88AB8076
:108DF00033464C33D2181388EB8052882A8165465B
:108E00006D1C4572491CC9B2A142D1D3174A002139
:108E1000204B9C3A8C00491CC9B213510C29F9D340
:108E2000007C002805D011490B7848788A78022BFD
:108E30000ED0154A002180320F2001F062FC012182
:108E40000520002249020007FDF77FFD0FB0F0BDAD
:108E5000074BC91C9B1F1818FCF790F901F002FE84
:108E6000642001F0A5F82FE5C60000203C13002087
:108E7000320D002048000020E0000020A01100205A
:108E8000983A0000CE00002000D02724CA0000201D
:108E9000C8000020FFFF010070470000FEB54149F7
:108EA0003F48086001F07EFD3F4800F0C9F83F4CA4
:108EB00020833D48801C00F0C3F860833A48001DC1
:108EC00000F0BEF8A083FF20394D1F30688028468F
:108ED00040300179E1710291E88E3649C0B20870E4
:108EE0000190E88F2071A88F6071A87AA070A8887F
:108EF000009060622889FCF7C1FB2F4A2F4BFCF7DA
:108F0000B7FA00F0F1FF00222D4BFCF7FFF9FCF758
:108F1000FBFB86B2A681EF8831463846FCF7E8F8BD
:108F2000E08101460098FCF7E3F871438EB27D20A2
:108F3000C00066817043FCF7A1FB224A224BFCF77C
:108F4000FFFAFCF7E1FB20827D20A6823946C000B3
:108F5000FCF7CEF86082E083688F207202990120CE
:108F6000002902D120710A212172002F01D1642130
:108F7000E980019A0F49432A01D943220A702084CB
:108F8000FCF7DEFEE082228A10491148FDF7A6FEBA
:108F90006888C2B2010A0FA000F0F4FDFEBD000017
:108FA000799A000844000020004F0008BC0000200F
:108FB0002C0D002000000020666666666666E63FAF
:108FC00000000840F853E3A59B843E40FF7F00006B
:108FD000B0140020CEEFD7CAB1EAC7A92DB7C0D7C9
:108FE000B2BBE3D7DC5625642E25640D0A000000D1
:108FF00070B586B014216846FCF7D9F801250F4EEC
:10900000ED03002229463046FDF79FFC0120002495
:10901000019002946946009503943046FDF7D4FB15
:109020000320019002946946009503943046FDF7B1
:10903000CBFB022000F0BCFF06B070BD0004005066
:109040000088704770470000F8B5044600206A4663
:109050001080194D55222A70AA226A700322AA7024
:10906000661DEE702A716971144A49008918AC7145
:109070002246E81DFCF782F8002007E029186A461E
:109080008978128889186A461180401CB042F5DB45
:10909000611DA81CFCF7CEFC014668460180291919
:1090A0000078C87168464078087221460931024844
:1090B00000F042FBF8BD0000F01300202C0D002052
:1090C00010B513490A8CCB8B9A4201D3D21A0A8469
:1090D000104A098CD2884A437D211018C9004843A0
:1090E0000D490968401AFCF7B5FA0C4A0C4BFCF71D
:1090F00027FAFCF7E5FA0B49884201DD4A4280185D
:10910000002800DA401808490968486110BD0000CD
:10911000BC0000202C0D002084000020F853E3A5A3
:109120009B843E40FF7F0000B0140020034A11687A
:10913000382389B2994301431160704700300140E0
:1091400010B5FDF70FFC10BD10B59AB0342168467C
:10915000FCF72DF814210DA8FCF729F81C2112A802
:10916000FCF725F81B4801680324E402A143C2145C
:1091700089180160FDF706FE17480169A1430161E6
:1091800006200090FF200130029001200390102063
:1091900004900220099040040B90000100240C90E0
:1091A0000A946846FDF7ECFF0F200D9003200E9007
:1091B0000F941094012111940DA8FDF7CFFE81208A
:1091C0001290032080041890149412A8FDF714FE46
:1091D0001AB010BD007000404010024010480168F5
:1091E000821511430160C1680E4A1140C1600168D7
:1091F0000D4A114001608168490849008160016899
:109200000122920491430160C168FD22120491433E
:10921000C160002101610649044888607047000070
:10922000001002400C40FF88F6FFF6FE00500008D8
:1092300000ED00E070B5026801239B07114C124D50
:10924000984203D0A04201D0A84203D17026B24375
:109250004E683243984203D0A04201D0A84204D1C4
:1092600003231B029A43CB681A4380239A430B695A
:109270001A4302608A68C262096881620121416101
:1092800070BD0000000801400014014010B5CB067D
:10929000DB0E0121046A99408C430462016A9A4002
:1092A0001143016210BD30B58468FF252D021B02F9
:1092B0001343AC430B432343836030BD8268702368
:1092C0009A430A4307210A438260704730B5026A15
:1092D000520852000262026A456883697024A343FF
:1092E0009C080B68A40023430224A2438C684560B9
:1092F0001443836149684163046230BD30B5026A3A
:1093000010239A430262036A456882697324240227
:10931000A2430C6824021443202293438A684560C8
:1093200012011A43846149688163026230BD30B51D
:10933000026AFF2301339A430262026A4568C369E5
:109340007024A3439C080B68A400234301246402F7
:10935000A2438C68456024021443C3614968C16319
:10936000046230BD30B5026A01231B039A430262D6
:10937000036A4568C26973242402A2430C6824026C
:1093800014430122520393438A68456012031A432F
:10939000C46149680164026230BD30B5036A046A81
:1093A0006408640004628469F025AC43120122431E
:1093B0000A24A3430B438261036230BD30B5036AC4
:1093C0001024A34303628469036A0F252D0312034B
:1093D000AC432243A024A3430901194382610162E3
:1093E00030BD000070B501F05BF80D4C0D4D6064B0
:1093F00002E001F055F86064A842FAD10020E08252
:109400002078002809D0012802D0022805D102E0E6
:10941000FCF7B2FC01E0FFF777F900F033FF70BD15
:10942000480000203001CADE10B5818CC90707D082
:1094300001684A6801235B049A43836A1A434A60BD
:10944000818C890707D501684A6801231B049A4368
:10945000C36A1A434A60818C490707D501684A6884
:1094600001239B049A43036B1A434A60818C0907CA
:1094700007D501684A680123DB039A43436B1A430B
:109480004A60818CC90607D50268916801231B03D5
:109490009943836B19439160818C890607D50168D4
:1094A0008A6801235B039A43C36B1A438A60818CE9
:1094B000490612D503685A6801210905046C8A43DC
:1094C00022435A60026C8A4207D102685168032322
:1094D0005B059943436C19435160818C090607D59C
:1094E00001684A680123DB04806C9A4302434A60A6
:1094F00010BD0000F8B500260446C667FDF72CFA3B
:10950000054620680068124F000709D501212B4647
:10951000002249052046009700F054FA00280DD19A
:109520002068006840070BD501212B4600228905E1
:109530002046009700F046FA002801D00320F8BD2D
:1095400020206067A067603426740020F8BD00000A
:10955000FFFFFF01F8B5184CC826E078002829D194
:109560006079002826D101206071144D686B0027B6
:1095700000281ED0686BC821081A15E01048E16861
:10958000405C616988470F480A21008848430E49BA
:109590000880E068401CE060E068C82800DBE76005
:1095A000696BC820401A761EE168814201D0002E06
:1095B000E4DC6771F8BD00003000002000000240CC
:1095C000640C0020CE000020DE00002070B5224C8C
:1095D000E07800283FD1207900283CD1012020717B
:1095E0001E4EF16900250906002933DA215662571B
:1095F00091420AD1F06940062CD5A079002829D0E3
:10960000A5712089401C208124E0A179002903D183
:10961000A0710A2000F0D3FC00202056CC21484342
:109620000F494218206912181279B262401C0022B8
:109630002061A256CC235A43895881420ADC256115
:109640002078401C207020780E2800D12570A0784A
:10965000401CA070257170BD300000200038014012
:109660003C01002010B5806A0022014640314A8347
:109670004A82FEF79AF910BD70B5846A606FA56FD3
:109680002168896800260906002906DA212804D104
:1096900052200653204600F047F8206880684006B4
:1096A00006D5222D04D15A200653204600F02CF86E
:1096B000E06F10210843E0672046FEF776F970BDA1
:1096C00010B501460968806A0968890614D4002229
:1096D0005A210A5201680A68FF2301339A430A603B
:1096E00001688A68520852008A6001688A684023CB
:1096F0009A438A6020218167FEF7F2FA10BD10B507
:10970000806AFEF7EEFA10BD01680A68FF23213374
:109710009A430A6001688A68520852008A602021D0
:10972000816700210166704701680A68C0239A4377
:109730000A6020214167704770B5164CE278002A14
:109740000CD12279002A09D10122E2700025C82912
:1097500003DC0222A256002A01DCE57070BD012361
:10976000E356CC2253430C4AD1500123E356CC2676
:1097700073439B180A460146181DFBF7FFFC6078EF
:10978000401C607060780E2800D16570A078401E83
:10979000A070E2E7300000203C010020F8B504464C
:1097A0002669A268E76932436669102000253E43B6
:1097B0002368324378491E68784F3E4016431E6046
:1097C00023685A6803263603B243E66832435A6078
:1097D0002368A2698B4201D0266A32439E680B2718
:1097E0003F02BE4316439E606D4E23686D4AB342EE
:1097F0000CD1D2689207920F06D0012A38D0022AE3
:1098000034D0032A20D11EE001201DE0664EB34271
:109810000AD1D2680C26324026D0042A28D0082A41
:1098200024D00C2A10D10EE08B420DD1D668032231
:109830009202164018D001229202B61A18D0B61A17
:1098400014D0964200D10820564A0126403A574F7C
:10985000F6038B4236D100280CD002280DD0042804
:1098600012D008281FD11CE00020EDE70220EBE712
:109870000420E9E7FDF728FC08E01068C00601D5E0
:10988000384605E04A4803E0FDF73EFC002873D067
:10989000626851005118814205D81103814202D3F8
:1098A00003E03046F4E7012566E0010E06025008A9
:1098B000002330185941FBF731FC03210902411AFA
:1098C0003C4A55E0E169B14232D1030000F081F930
:1098D00009070A0D06250606062B0600E3E7FDF735
:1098E000F3FB1CE0FDF700FC19E010686168C0069E
:1098F00002D54808304A01E0304A48088018FBF792
:10990000F7FB80B201462E4A10399142CBD8511C48
:1099100001400007400F08432CE0FDF7F5FB6168AC
:1099200040004A08EAE76168012248081204E5E7B6
:10993000030000F04EF909070A0D06260606062C5C
:109940000600B0E7FDF7C0FB1DE0FDF7CDFB1AE018
:1099500010686168C00602D54808C01902E01448C2
:109960004A081018FBF7C4FB80B20146144A1039AC
:10997000914298D82168C860002020666066284619
:10998000F8BDFDF7C1FB61684A088018EAE7616825
:1099900048088019E6E7000000480040F369FFEF3F
:1099A00000380140401002400044004000093D00E2
:1099B0000024F400FFFC0F0000127A000048E801C8
:1099C000EFFF0000FFB581B017460E4604460A9D22
:1099D00009E0681C07D0FCF7BFFF0499401AA842B1
:1099E0000CD8002D0AD02068C1693046884318D0B1
:1099F0000020B842EDD0002005B0F0BD206801681D
:109A0000FF22A13291430160206881684908490022
:109A1000816020206067A0670020603420740320EC
:109A2000EAE70120E5E7000010B5044910200968C5
:109A300008620248FDF7BAFF10BD0000741500204F
:109A400001490D20887070473000002010B507488C
:109A50000A22418A51434184FEF7D0FCFEF7ECFD17
:109A6000C82203490348FEF7DFF810BDBC00002000
:109A7000640C002074150020F8B53D4C00232178BB
:109A80003C4A1D46082910D0072945D006294ED04A
:109A9000052950D0042951D0032952D0002954D08F
:109AA000012956D0022958D059E0A17800264A1F32
:109AB00004E0304FBF5DFB189BB2761C9642F8DB8A
:109AC000667927799A195118E3786278C918891844
:109AD000C9194018C0071AD0012E14D0022E16D171
:109AE00025482449C018FBF749FB00F0BBFF642060
:109AF00000F05EFABFF34F8F21492048C860BFF3E2
:109B00004F8F00BFFDE759081046FFF79DFA2570FB
:109B1000E570A570A571F8BDA1795054491CC8B273
:109B2000A071A178491F8842F5D1082001E060703A
:109B300007202070F8BDE0700620FAE7607105206C
:109B4000F7E7A070E5700420F3E7552807D101205E
:109B5000EFE7AA2803D10220EBE7032803D0257002
:109B6000E570A570F8BD032020702071F8BD0000DD
:109B7000B30000208C1300202C0D00200400FA05F7
:109B800000ED00E00FB410B503A9044B044A02989D
:109B900000F002F910BC08BC04B01847E1A70008A7
:109BA000FC0000202021020C01D010211046020AE6
:109BB00001D010460839020901D01046091F820859
:109BC00001D01046891E420801D0881E7047081A2D
:109BD000704730B47446641E2578641CAB4200D2D2
:109BE0001D46635D5B00E31830BC184702E008C8FF
:109BF000121F08C1002AFAD170477047002001E007
:109C000001C1121F002AFBD1704708B50021684628
:109C100001706B46012202212C2000F081FD0221FF
:109C2000684601706B4601222C2000F079FD08BDCA
:109C300038B504466D20694608706B460122074915
:109C40002E2000F06DFD0649002C01D0054A00E0F1
:109C5000054A2E2000F04AFD38BD0000060800002D
:109C600006180000070600000716000038B5044675
:109C70006B4602220021362000F018FCB32123009D
:109C8000FFF7A7FF0E0F08153A3A3A3A1C273A3A5F
:109C90002F34483A00216846017040784108490055
:109CA00014E06946087880088000401C04E069469A
:109CB000087880088000801C08701DE068460278E3
:109CC0000A40483202704178802001436846417062
:109CD00012E0684602780A40027040784106490E58
:109CE000F4E7694648780221084303E0694648786A
:109CF000FD210840694648706B460122002136204C
:109D000000F00EFD012200AB11463620013300F0B9
:109D100007FD38BD69460878CF21084069462030E4
:109D2000CAE708B5032168464170012101706B46FE
:109D300002220021362000F0F3FC0122D20306218A
:109D40002D2000F0D3FC012000F032F90120FFF7B4
:109D50008DFF08BD08B5020A69464A7008706B4657
:109D6000022204212D2000F0DBFC0320694608704C
:109D70006B46012206212D2000F0D2FC002069460E
:109D800008706B46012206212D2000F0C9FC0A2133
:109D90002D2000F071FB08BDFFB58DB004460025F5
:109DA00006E025280AD0109A0F999047641C6D1C74
:109DB00020780028F5D1284611B0F0BD00270121F8
:109DC000484A009700E00743641C23780846203B7C
:109DD00098401042F7D120782E2817D1042007434D
:109DE0006078641C2A280CD10E98641C02C800916B
:109DF0000E900BE000990A22514330394018641C40
:109E000000902078014630390929F3D920780028BC
:109E1000D1D0642808D0692806D075281ED0109AA1
:109E20000F9990476D1C5BE00A200E99019001C9C3
:109E30000E91002802DA40422D2102E0390504D5B6
:109E40002B216A461172012103E0F90704D0202179
:109E5000F7E70BAE0B910DE00021FAE70A200E990F
:109E6000019001C90E91F7E70199FBF741F93031F3
:109E7000761E31700028F7D103A8801B2030019096
:109E8000780701D5009801E00120009001998842EF
:109E900001DD401A00E000200027009006E002A843
:109EA000109AC05D0F9990476D1C7F1C0B988742DC
:109EB000F5DB04E0109A30200F9990476D1C009953
:109EC000481E00900029F5DC05E03078109A761CD9
:109ED0000F9990476D1C0199481E01900029F4DCF0
:109EE000641C65E709280100F8B54A002B4B520DA8
:109EF000D6182B4A0C460546142E2BDA002E12DA01
:109F0000284BFBF703FA00221346FBF729FD40D24A
:109F1000002C03DA0124E40700253AE02046284318
:109F200037D0214C14E0214F0B46F7403B402B43E8
:109F300031D01C4BFBF7EAF900221346FBF710FD6A
:109F400027D2002C03DD01200005F0400419BC439A
:109F500000251EE0332E1EDC33460027143BFF4352
:109F6000DF40384217D00F4BFBF77AFA0022134636
:109F7000FBF7F6FC0DD2002C0ADD142E0CD0342099
:109F8000811B012088404019A84200D2641C05466C
:109F9000BD4321462846F8BD641CF9E701FCFFFFDC
:109FA0009C7500883CE4377E0000F03FFFFF0F0007
:109FB0007D2110B5C900484300F001F810BD002113
:109FC00040E000BF00BF00BF00BF00BF00BF00BF38
:109FD00000BF00BF00BF00BF00BF00BF00BF00BF89
:109FE00000BF00BF00BF00BF00BF00BF00BF00BF79
:109FF00000BF00BF00BF00BF00BF00BF00BF00BF69
:10A0000000BF00BF00BF00BF00BF00BF00BF00BF58
:10A0100000BF00BF00BF00BF00BF00BF00BF00BF48
:10A0200000BF00BF00BF00BF00BF00BF00BF00BF38
:10A0300000BF00BF00BF00BF00BF00BF00BF00BF28
:10A0400000BF491C8142BCD370470000FEB50446E6
:10A050000020019000906079734940000E5A6178A9
:10A060002578491E7148CFB20163042D77D0072DA2
:10A0700075D000210291217801736C49E3790122A6
:10A0800092058969002B6CD0914381616748217AE0
:10A090004173217A82698907890B0A438261002111
:10A0A000042000F02EFB324661492E2000F01EFBFA
:10A0B0003846FFF7BDFD5F4E0522705D81004018F8
:10A0C0005D49431807212B2000F02AFB5B490298C9
:10A0D00001220B180B21282000F022FB705D58494B
:10A0E00080000A580C21282000F00BFBE07955492C
:10A0F00080004018A1794900425A0221272000F02F
:10A10000F5FA51487E00825B0421272000F0EEFA28
:10A11000E079002829D0A07804282CD0282069468E
:10A12000087220220621272000F0E0FA02AB01226B
:10A130002621272000F0F4FA444938014018E1783C
:10A14000890042580821272000F0DBFAA17A601C20
:10A15000627A0902114313D016E000E001E0012108
:10A1600088E71143F608816190E7642206212720E1
:10A1700000F0BCFAE0E71020694608720246D1E719
:10A1800033490172090A4172417A007A0A02024394
:10A190002021272000F0AAFA2E4F0C2123203A6814
:10A1A00000F0AFFAF01982880421232000F09EFA13
:10A1B000A07900280BD0E07927490122431800211B
:10A1C000212000F0ADFA03200190012000902A0721
:10A1D000120F10010243607800218007000B024338
:10A1E0000198000502430098400402432079C0060C
:10A1F000400902436079C00602431F2000F081FA43
:10A20000A07861780123084302040848DB03026157
:10A21000E179490319430A4302610021082000F053
:10A2200070FA0020FEBD000030AB000800010020E5
:10A2300004280000D8AA0008010000201F00002008
:10A24000E0AA000800AB00080CAB000810AB000847
:10A2500041100000F8AA00082100002038B50C4683
:10A2600007498A8B002102432C2000F03FFA684600
:10A2700004706B46012206212C2000F051FA38BDF3
:10A280000001002010B5FFF7C0FC10BD10B504465A
:10A290000421362000F0F0F80121C902002C01D081
:10A2A000084300E0884302460421362000F029FAE2
:10A2B00010BD000038B540206946087000210E200E
:10A2C00000F0DAF80446002211460E2000F019FAD8
:10A2D0006B46012200210D2000F022FA074A0021DE
:10A2E0000F2000F00EFA00F0E7F9224600210E20C0
:10A2F00000F007FA02480021017338BDF8FF272457
:10A30000200100207CB505460420694608704B4CAE
:10A310000020607521462031206348710873A083B6
:10A320006063A06300F0BCF8454E206002E000F0DE
:10A33000B7F82060B042FAD10020FFF797FC4148FF
:10A340000078242801D9243806E00621FAF7D0FE47
:10A350000622101A40010843020601040A430102C2
:10A360000A43024300211E2000F0CBF96B46012274
:10A370000021242000F0D4F91E20FFF7EBFC86B268
:10A38000300AA0730420FFF7E5FC0006000E0DD094
:10A3900002206946087101AB012212212D2000F034
:10A3A000BFF9A08B012109030843A08300F078F8CE
:10A3B00020600620FFF7CEFC60600720FFF7CAFC94
:10A3C000A060F006C00E207501D110202075C0B22B
:10A3D00000F0E2F9E80707D0FFF7A3FCA08B01210A
:10A3E000C9020843A0830AE00521362000F02EF8B8
:10A3F0001549084002460521362000F077F9012072
:10A40000FFF734FC0021042000F036F8A0610021A1
:10A41000262000F031F81521890308430246002167
:10A42000262000F06EF900222621362000F05EF989
:10A4300000F036F8206000207CBD00000001002004
:10A440003001CADE00000020FFFD000038B5094CD5
:10A4500089B280B26B46022200F028F8002806D1AB
:10A4600068464078010268460078081884B22046A1
:10A4700038BD0000FFFF000038B50024E44389B276
:10A4800080B26B46042200F011F8002806D10321A7
:10A490006846435C2202D418491EFAD5204638BDCE
:10A4A00010B500210846FFF7E7FF10BD38B50029B9
:10A4B00009D0402420436C462070C8B27F2906D8BA
:10A4C000607002200AE069460870012006E08024DE
:10A4D00020436C466070C809A0700320694600F0F4
:10A4E0009BFA38BD10B5144603460A462146112092
:10A4F000FFF7DCFF10BD10B5034605220021152033
:10A50000FFF7D4FF10BD10B501210620FFF7B4FFFF
:10A5100010BD10B50346052200211720FFF7C6FF26
:10A5200010BD38B5054600206946087000F0C4F833
:10A53000FF2401342246002D01D003221202002103
:10A540000D2000F0D3F8002D13D06B46012203211B
:10A550000F20FFF7ABFF68460078000709D5FFF72B
:10A56000A9FE224600210D2000F0C0F80020C043C3
:10A5700038BD002038BD10B5024601210A2000F088
:10A58000C0F810BD10B5044600211A20FFF774FF73
:10A59000000D22030005120B024300211A2000F0D7
:10A5A000B0F810BD10B5024602492E2000F09EF80A
:10A5B00010BD000004180000F8B505466B460122E6
:10A5C00003210420FFF772FF0126114C3607002DEE
:10A5D0000DD02A4600210C2000F088F86946087842
:10A5E0001021084369460870A069304307E06946B6
:10A5F0000878EF21084069460870A069B0430B460F
:10A60000A06101220321042000F08AF8F8BD0000B7
:10A610000001002010B502460021182000F066F865
:10A6200010BD0000F8B50746002568460570B8075C
:10A63000204C2E4600280ADA8020694608706B46B6
:10A64000012200210D2000F06BF801202073F80793
:10A650006946087821D006210843694608706B4690
:10A66000012200210D2000F05BF803210F20FFF7ED
:10A67000EDFE8121C900084219D0402069460870CA
:10A680006B46012200210D2000F04AF80020FFF760
:10A69000FDFD00252673ED4309E0022108436946CC
:10A6A00008706B46012200210D2000F039F8284681
:10A6B000F8BD0000200100201CB56B4601220321DB
:10A6C0000F20FFF7F3FE684600784022C1091040D2
:10A6D000C9014000814208D0012069460871024644
:10A6E00001AB03210D2000F01BF81CBD08B56B4623
:10A6F0001A70120A5A7089B280B2022200F010F861
:10A7000008BD38B500236C46E254120A5B1C042BCA
:10A71000FADB89B280B22346042200F001F838BD8A
:10A7200038B58024002909D0C02528436D462870FB
:10A73000C8B27F2907D86870022009E02043694623
:10A740000870012004E020436870C809A870032045
:10A75000694600F09DF938BD10B514460123121862
:10A760009B029A4202D90020C04310BD0B46821EB4
:10A7700021460920FFF7D4FF002010BD10B5054A7F
:10A780008905126901430A4300210820FFF7B9FF38
:10A79000002010BD0001002038B504466B460122A0
:10A7A0000E212B20FFF782FE68460078E106400963
:10A7B0004001C90E0143684601706B4601220E211B
:10A7C0002B20FFF7ADFF38BD10B5002142541C0609
:10A7D000120A22431B0A491C0429F7DB10BD0000A2
:10A7E00013B501231A4669460248FDF77BFA009823
:10A7F0001CBD000074150020FCF7BCF8FEF7A4FC9B
:10A80000FDF7FCFDFDF70EFE40494148002522C042
:10A8100005608561C5613F490562C1600838FCF784
:10A82000DFF9FDF709FFFDF7A3FEFDF7B3FDFDF727
:10A83000C1FE052601223607D1033046FCF785F814
:10A84000FEF72CFBFDF7A6FCFBF74AF9FBF722F914
:10A850000721B015FFF702FDFFF714FD2E4C0A216A
:10A86000608A01224843608411033046FCF76DF88A
:10A870002748C8222949C430FDF7D6F9284F294E68
:10A88000E07800283ED0E07900283BD0FEF75CFC61
:10A89000E570FBF73DFB20700F280AD90122110358
:10A8A0003046FCF752F8FEF79DFD00220121090316
:10A8B00009E0012251033046FCF747F8FEF792FD0C
:10A8C0000022012149033046FCF73FF8FDF794FBD5
:10A8D000608C002801D0401E60841348618C007891
:10A8E0000843CDD13878002801D00328C8D14021B1
:10A8F0003046FCF725F80028C2D101210846FCF7B4
:10A9000061FABDE7FDF778FBBAE70000007C004084
:10A91000B0140020FFFF0000BC000020640C0020E9
:10A920005A000020000400503600002010B586B008
:10A930001748FCF7DAF814216846FAF738FC15488E
:10A940000090032001900020029005206946000736
:10A95000FBF73AFF69461048FBF736FF69460F4898
:10A96000FBF732FF01210846FCF72CFAFF240134E3
:10A970002046FCF7FFF90A490868042210430860E2
:10A980002046FCF707FAFCF70DFA06B010BD0000F0
:10A99000B0140020FFFF0000000400500008005029
:10A9A0000070004010B50122920218491848FBF7C8
:10A9B0000DF91648174902888A4226D001800421E1
:10A9C0008180FF21F531C1800A21018100211E22F1
:10A9D0004181D24382810122C2810184018241826C
:10A9E0008182C182018381834323C386022303873B
:10A9F000782343878287C287024640329180118440
:10AA000051849184C18300F02DF810BD2C0D0020DD
:10AA100000FC0008AA550000F0B58C460025102661
:10AA2000052109078E620E4C08E067467F5DE760EE
:10AA3000A768FF07FCD0E7681F706D1C8542F4DB38
:10AA40000020074606E0E760A568ED07FCD0E56852
:10AA50001D54401C9042F6D38E610020F0BD0000D2
:10AA60000030014070B572B60124074DA4022146A2
:10AA70002846FBF791F8002804D0224603492846CF
:10AA8000FBF72EF962B670BD00FC00082C0D00200B
:10AA9000F0B50025102605279C463F070B46BE62F1
:10AAA0000C4C06E0595DE160A168C907FCD0E16883
:10AAB0006D1C8542F6DB002007E06146095CE16021
:10AAC000A168C907FCD0E168401C9042F5D3BE6183
:10AAD0000020F0BD00300140000001020304000529
:10AAE000405C0000A05C0400C06C0800805C0400B6
:10AAF000E03F1E00E07D1E0007A9022570889B88AC
:10AB00000A001600010006000100020087008D0007
:10AB10002D001A3152001A339A001A351D011A37C6
:10AB20006B003B31BE003B335E013B3596023B3749
:10AB3000000099599959EB518F421E45142E0080FF
:10AB4000EB51F5283333E13A703DE13AC235852BBC
:10AB5000C2353333C235C235AE47E13A5138A3303E
:10AB60005138000000000000000001020304060745
:10AB70000809030406080C1018203000000000012A
:10AB800002030400A4AB0008000000200001000044
:10AB9000EC9B0008A4AC000800010020A0190000F4
:10ABA000FC9B000800070400091E08054008260950
:10ABB0001040085608054008261D040008BE1D0464
:10ABC0000008BED8BC401008010000000000C842C8
:10ABD0000000000000000000000000000000000075
:10ABE0000000000000000000000000000100000064
:10ABF0000000000000000000000000000000000055
:10AC00008C0A0000000000000000000000000000AE
:10AC10000000000000000000000000000000000034
:10AC20000000000000000000000000000000000024
:10AC30000000000000000000000000000000000014
:10AC400000000000000000000000000002021400EC
:10AC5000090901020081000000000000010000005D
:10AC600000000000000000000000000000000000E4
:10AC700000000000000000000000000000000000D4
:10AC800000000000000000000000000000000000C4
:10AC90000000000000000000000000000000200094
:04ACA00000000000B0
:04000005080050C1DE
:00000001FF
